:020000040000FA
:10000000031714309E0008309F000313831600303E
:100010008700163085002030860010309F00831244
:10002000870185018601A801A501352041204130C5
:100030009F002B20A100833062204D309F002B2099
:10004000A100C33062206D309F002B20A1009730AB
:100050006220B62017280000000000000000000009
:100060009F149F1C31281E08080007148F20383069
:1000700087008F200C3087008F20063087008F206C
:10008000080080305C20583054203A305420C03072
:100090005C20593054203A30542094305C205A303F
:1000A00054203A3054200800A50095200514250856
:1000B00087008F2005100800A500952025088700DF
:1000C0008F2008005C20A201A301A4017120240854
:1000D000AA2054202308AA2054202208AA20542011
:1000E0000800003003112106031908000A3003112B
:1000F000220203197E28A103A20A7128A201A30AE1
:1001000009300311230203198720A1037128A301D9
:10011000A40A0930031124020319A40A08000616D0
:10012000000000000000000006128316FF30870068
:100130008312851600000000061600000000000073
:1001400000000612871B9C2885128316003087004A
:10015000831208008207303431343234333434347B
:10016000353436343734383439340800A60BB628E1
:06017000A70BB6280800F1
:02400E00D430AC
:00000001FF
